BL51 BANKED LINKER/LOCATER V6.22                                                        01/21/2022  11:45:08  PAGE 1


BL51 BANKED LINKER/LOCATER V6.22, INVOKED BY:
D:\KEIL_V5\C51\BIN\BL51.EXE STARTUP.obj, main.obj, LCD.obj, sys.obj, font.obj, touch.obj TO ceshi RAMSIZE (256)


MEMORY MODEL: LARGE WITH FLOATING POINT ARITHMETIC


INPUT MODULES INCLUDED:
  STARTUP.obj (?C_STARTUP)
  main.obj (MAIN)
  LCD.obj (LCD)
  sys.obj (SYS)
  font.obj (FONT)
  touch.obj (TOUCH)
  D:\KEIL_V5\C51\LIB\C51FPL.LIB (?C?FPADD)
  D:\KEIL_V5\C51\LIB\C51FPL.LIB (?C?FPMUL)
  D:\KEIL_V5\C51\LIB\C51FPL.LIB (?C?FPDIV)
  D:\KEIL_V5\C51\LIB\C51FPL.LIB (?C?FPCMP)
  D:\KEIL_V5\C51\LIB\C51FPL.LIB (?C?FCAST)
  D:\KEIL_V5\C51\LIB\C51FPL.LIB (?C?CASTF)
  D:\KEIL_V5\C51\LIB\C51FPL.LIB (?C?FPGETOPN)
  D:\KEIL_V5\C51\LIB\C51L.LIB (?C_INIT)
  D:\KEIL_V5\C51\LIB\C51L.LIB (?C?CLDPTR)
  D:\KEIL_V5\C51\LIB\C51L.LIB (?C?IMUL)
  D:\KEIL_V5\C51\LIB\C51L.LIB (?C?UIDIV)
  D:\KEIL_V5\C51\LIB\C51L.LIB (?C?IILDX)
  D:\KEIL_V5\C51\LIB\C51L.LIB (?C?ISTPTR)
  D:\KEIL_V5\C51\LIB\C51L.LIB (?C?LMUL)
  D:\KEIL_V5\C51\LIB\C51L.LIB (?C?ULDIV)
  D:\KEIL_V5\C51\LIB\C51L.LIB (?C?LNEG)
  D:\KEIL_V5\C51\LIB\C51L.LIB (?C?ULCMP)
  D:\KEIL_V5\C51\LIB\C51L.LIB (?C?LSTXDATA)
  D:\KEIL_V5\C51\LIB\C51L.LIB (?C?LSTKXDATA)


LINK MAP OF MODULE:  ceshi (?C_STARTUP)


            TYPE    BASE      LENGTH    RELOCATION   SEGMENT NAME
            -----------------------------------------------------

            * * * * * * *   D A T A   M E M O R Y   * * * * * * *
            REG     0000H     0008H     ABSOLUTE     "REG BANK 0"
            IDATA   0008H     0001H     UNIT         ?STACK

            * * * * * * *  X D A T A   M E M O R Y  * * * * * * *
            XDATA   0000H     0082H     UNIT         _XDATA_GROUP_
            XDATA   0082H     0016H     UNIT         ?XD?LCD
            XDATA   0098H     0010H     UNIT         ?XD?TOUCH
            XDATA   00A8H     0001H     UNIT         ?XD?MAIN

            * * * * * * *   C O D E   M E M O R Y   * * * * * * *
            CODE    0000H     0003H     ABSOLUTE     
            CODE    0003H     1370H     UNIT         ?CO?FONT
            CODE    1373H     0CA7H     UNIT         ?PR?TOUCH_ADJUST?TOUCH
            CODE    201AH     0604H     UNIT         ?C?LIB_CODE
            CODE    261EH     01F7H     UNIT         ?PR?_DRAW_CIRCLE?LCD
            CODE    2815H     01F2H     UNIT         ?PR?XIANSHI?MAIN
BL51 BANKED LINKER/LOCATER V6.22                                                      01/21/2022  11:45:08  PAGE 2


            CODE    2A07H     01EBH     UNIT         ?PR?_LCD_DRAWLINE?LCD
            CODE    2BF2H     019EH     UNIT         ?PR?_LCD_SHOWCHAR?LCD
            CODE    2D90H     0170H     UNIT         ?PR?LCD_INIT?LCD
            CODE    2F00H     0157H     UNIT         ?PR?_ADS_READ_XY?TOUCH
            CODE    3057H     0131H     UNIT         ?PR?_READ_ADS2?TOUCH
            CODE    3188H     0115H     UNIT         ?PR?SHOWIMAGE?MAIN
            CODE    329DH     0103H     UNIT         ?PR?CONVERT_POS?TOUCH
            CODE    33A0H     00E8H     UNIT         ?PR?_DROW_TOUCH_POINT?TOUCH
            CODE    3488H     00E1H     UNIT         ?PR?_LCD_SHOWNUM?LCD
            CODE    3569H     00D9H     UNIT         ?PR?POINT?TOUCH
            CODE    3642H     00CFH     UNIT         ?PR?_SHOWHANZI?LCD
            CODE    3711H     00AAH     UNIT         ?PR?_LCD_DRAWRECTANGLE?LCD
            CODE    37BBH     00A1H     UNIT         ?PR?_LCD_SHOWSTRING?LCD
            CODE    385CH     008CH     UNIT         ?C_C51STARTUP
            CODE    38E8H     0086H     UNIT         ?PR?_LCD_FILL?LCD
            CODE    396EH     0082H     UNIT         ?PR?_LCD_SHOW2NUM?LCD
            CODE    39F0H     007BH     UNIT         ?PR?READ_TP_ONCE?TOUCH
            CODE    3A6BH     006BH     UNIT         ?CO?TOUCH
            CODE    3AD6H     0063H     UNIT         ?PR?_READ_ADS?TOUCH
            CODE    3B39H     005EH     UNIT         ?PR?JIANCE?MAIN
            CODE    3B97H     005CH     UNIT         ?PR?_LCD_CLEAR?LCD
            CODE    3BF3H     0052H     UNIT         ?PR?_LCD_DRAWPOINT?LCD
            CODE    3C45H     004CH     UNIT         ?PR?_LCD_DRAWPOINT_BIG?LCD
            CODE    3C91H     0049H     UNIT         ?C_INITSEG
            CODE    3CDAH     0049H     UNIT         ?PR?_MYPOW?LCD
            CODE    3D23H     003AH     UNIT         ?PR?_ADDRESS_SET?LCD
            CODE    3D5DH     0033H     UNIT         ?PR?MAIN?MAIN
            CODE    3D90H     0029H     UNIT         ?CO?MAIN
            CODE    3DB9H     0026H     UNIT         ?PR?_DELAYMS?SYS
            CODE    3DDFH     0022H     UNIT         ?PR?READFROMCHARFROM7843?TOUCH
            CODE    3E01H     001AH     UNIT         ?PR?_WRITECHARTO7843?TOUCH
            CODE    3E1BH     0017H     UNIT         ?PR?_ADS_READ_AD?TOUCH
            CODE    3E32H     0014H     UNIT         ?PR?_LCD_WR_DATA?LCD
            CODE    3E46H     000EH     UNIT         ?PR?_LCD_WR_REG_DATA?LCD
            CODE    3E54H     000BH     UNIT         ?PR?_LCD_WRIT_BUS?LCD
            CODE    3E5FH     000BH     UNIT         ?PR?_LCD_WR_REG?LCD
            CODE    3E6AH     0009H     UNIT         ?PR?SPISTAR?TOUCH
            CODE    3E73H     0006H     UNIT         ?PR?TPSTATE?TOUCH
            CODE    3E79H     0005H     UNIT         ?PR?_LCD_WR_DATA8?LCD
            CODE    3E7EH     0002H     UNIT         ?CO?LCD



OVERLAY MAP OF MODULE:   ceshi (?C_STARTUP)


SEGMENT                                  XDATA_GROUP
  +--> CALLED SEGMENT                  START    LENGTH
------------------------------------------------------
?C_C51STARTUP                          -----    -----
  +--> ?PR?MAIN?MAIN
  +--> ?C_INITSEG

?PR?MAIN?MAIN                          -----    -----
  +--> ?PR?SPISTAR?TOUCH
  +--> ?PR?LCD_INIT?LCD
  +--> ?PR?_LCD_CLEAR?LCD
BL51 BANKED LINKER/LOCATER V6.22                                                      01/21/2022  11:45:08  PAGE 3


  +--> ?PR?SHOWIMAGE?MAIN
  +--> ?PR?JIANCE?MAIN

?PR?LCD_INIT?LCD                       -----    -----
  +--> ?PR?_LCD_WR_REG_DATA?LCD
  +--> ?CO?LCD
  +--> ?PR?_LCD_SHOWSTRING?LCD
  +--> ?PR?_LCD_SHOWNUM?LCD
  +--> ?PR?_LCD_SHOW2NUM?LCD
  +--> ?PR?_LCD_DRAWPOINT_BIG?LCD
  +--> ?PR?_LCD_DRAWRECTANGLE?LCD
  +--> ?PR?_DRAW_CIRCLE?LCD
  +--> ?PR?_DELAYMS?SYS
  +--> ?PR?_LCD_WR_REG?LCD
  +--> ?PR?_LCD_WR_DATA?LCD

?PR?_LCD_WR_REG_DATA?LCD               -----    -----
  +--> ?PR?_LCD_WR_REG?LCD
  +--> ?PR?_LCD_WR_DATA?LCD

?PR?_LCD_WR_REG?LCD                    -----    -----
  +--> ?PR?_LCD_WRIT_BUS?LCD

?PR?_LCD_WR_DATA?LCD                   -----    -----
  +--> ?PR?_LCD_WRIT_BUS?LCD

?PR?_LCD_SHOWSTRING?LCD                0043H    0007H
  +--> ?PR?_LCD_CLEAR?LCD
  +--> ?PR?_LCD_SHOWCHAR?LCD

?PR?_LCD_CLEAR?LCD                     004AH    0003H
  +--> ?PR?_ADDRESS_SET?LCD
  +--> ?PR?_LCD_WR_DATA8?LCD

?PR?_ADDRESS_SET?LCD                   0063H    0008H
  +--> ?PR?_LCD_WR_REG?LCD
  +--> ?PR?_LCD_WR_DATA?LCD

?PR?_LCD_WR_DATA8?LCD                  -----    -----
  +--> ?PR?_LCD_WRIT_BUS?LCD

?PR?_LCD_SHOWCHAR?LCD                  004FH    000CH
  +--> ?PR?_ADDRESS_SET?LCD
  +--> ?CO?FONT
  +--> ?PR?_LCD_WR_DATA?LCD
  +--> ?PR?_LCD_DRAWPOINT?LCD

?PR?_LCD_DRAWPOINT?LCD                 -----    -----
  +--> ?PR?_ADDRESS_SET?LCD
  +--> ?PR?_LCD_WR_DATA?LCD

?PR?_LCD_SHOWNUM?LCD                   0043H    000CH
  +--> ?PR?_MYPOW?LCD
  +--> ?PR?_LCD_SHOWCHAR?LCD

?PR?_MYPOW?LCD                         004FH    0006H

BL51 BANKED LINKER/LOCATER V6.22                                                      01/21/2022  11:45:08  PAGE 4


?PR?_LCD_SHOW2NUM?LCD                  0000H    0009H
  +--> ?PR?_MYPOW?LCD
  +--> ?PR?_LCD_SHOWCHAR?LCD

?PR?_LCD_DRAWPOINT_BIG?LCD             -----    -----
  +--> ?PR?_LCD_FILL?LCD

?PR?_LCD_FILL?LCD                      000AH    000CH
  +--> ?PR?_ADDRESS_SET?LCD
  +--> ?PR?_LCD_WR_DATA?LCD

?PR?_LCD_DRAWRECTANGLE?LCD             0000H    0008H
  +--> ?PR?_LCD_DRAWLINE?LCD

?PR?_LCD_DRAWLINE?LCD                  0047H    001CH
  +--> ?PR?_LCD_DRAWPOINT?LCD

?PR?_DRAW_CIRCLE?LCD                   0000H    000AH
  +--> ?PR?_LCD_DRAWPOINT?LCD

?PR?SHOWIMAGE?MAIN                     0000H    0006H
  +--> ?PR?_LCD_CLEAR?LCD
  +--> ?PR?XIANSHI?MAIN
  +--> ?PR?_ADDRESS_SET?LCD
  +--> ?PR?JIANCE?MAIN
  +--> ?CO?FONT
  +--> ?PR?_LCD_WR_DATA8?LCD

?PR?XIANSHI?MAIN                       0006H    0004H
  +--> ?PR?_SHOWHANZI?LCD
  +--> ?CO?MAIN
  +--> ?PR?_LCD_SHOWSTRING?LCD
  +--> ?PR?_LCD_SHOWNUM?LCD

?PR?_SHOWHANZI?LCD                     000AH    000AH
  +--> ?CO?FONT
  +--> ?PR?_ADDRESS_SET?LCD
  +--> ?PR?_LCD_WR_DATA?LCD

?PR?JIANCE?MAIN                        -----    -----
  +--> ?PR?TPSTATE?TOUCH
  +--> ?PR?_LCD_CLEAR?LCD
  +--> ?PR?POINT?TOUCH
  +--> ?PR?TOUCH_ADJUST?TOUCH
  +--> ?PR?_DELAYMS?SYS

?PR?POINT?TOUCH                        0006H    0004H
  +--> ?PR?CONVERT_POS?TOUCH
  +--> ?CO?TOUCH
  +--> ?PR?_LCD_SHOWSTRING?LCD
  +--> ?PR?_LCD_SHOWNUM?LCD
  +--> ?PR?_LCD_DRAWPOINT_BIG?LCD

?PR?CONVERT_POS?TOUCH                  000AH    0001H
  +--> ?PR?_READ_ADS2?TOUCH

?PR?_READ_ADS2?TOUCH                   0048H    000EH
BL51 BANKED LINKER/LOCATER V6.22                                                      01/21/2022  11:45:08  PAGE 5


  +--> ?PR?_READ_ADS?TOUCH

?PR?_READ_ADS?TOUCH                    0056H    0008H
  +--> ?PR?_ADS_READ_XY?TOUCH

?PR?_ADS_READ_XY?TOUCH                 005EH    0024H
  +--> ?PR?_ADS_READ_AD?TOUCH

?PR?_ADS_READ_AD?TOUCH                 -----    -----
  +--> ?PR?_WRITECHARTO7843?TOUCH
  +--> ?PR?READFROMCHARFROM7843?TOUCH

?PR?TOUCH_ADJUST?TOUCH                 0006H    003DH
  +--> ?PR?_LCD_CLEAR?LCD
  +--> ?PR?READ_TP_ONCE?TOUCH
  +--> ?PR?_DROW_TOUCH_POINT?TOUCH
  +--> ?CO?TOUCH
  +--> ?PR?_LCD_SHOWSTRING?LCD
  +--> ?PR?_LCD_SHOWNUM?LCD

?PR?READ_TP_ONCE?TOUCH                 0043H    0005H
  +--> ?PR?_READ_ADS2?TOUCH
  +--> ?PR?_DELAYMS?SYS

?PR?_DROW_TOUCH_POINT?TOUCH            0043H    0004H
  +--> ?PR?_LCD_DRAWLINE?LCD
  +--> ?PR?_LCD_DRAWPOINT?LCD



SYMBOL TABLE OF MODULE:  ceshi (?C_STARTUP)

  VALUE           TYPE          NAME
  ----------------------------------

  -------         MODULE        ?C_STARTUP
  C:385CH         SEGMENT       ?C_C51STARTUP
  I:0008H         SEGMENT       ?STACK
  C:0000H         PUBLIC        ?C_STARTUP
  D:00E0H         SYMBOL        ACC
  D:00F0H         SYMBOL        B
  D:0083H         SYMBOL        DPH
  D:0082H         SYMBOL        DPL
  N:0000H         SYMBOL        IBPSTACK
  N:0100H         SYMBOL        IBPSTACKTOP
  N:0080H         SYMBOL        IDATALEN
  C:385FH         SYMBOL        IDATALOOP
  N:0000H         SYMBOL        PBPSTACK
  N:0100H         SYMBOL        PBPSTACKTOP
  N:0000H         SYMBOL        PDATALEN
  N:0000H         SYMBOL        PDATASTART
  N:0000H         SYMBOL        PPAGE
  N:0000H         SYMBOL        PPAGEENABLE
  D:00A0H         SYMBOL        PPAGE_SFR
  D:0081H         SYMBOL        SP
  C:385CH         SYMBOL        STARTUP1
  N:0000H         SYMBOL        XBPSTACK
BL51 BANKED LINKER/LOCATER V6.22                                                      01/21/2022  11:45:08  PAGE 6


  N:0000H         SYMBOL        XBPSTACKTOP
  N:0000H         SYMBOL        XDATALEN
  N:0000H         SYMBOL        XDATASTART
  C:0000H         LINE#         126
  C:385CH         LINE#         133
  C:385EH         LINE#         134
  C:385FH         LINE#         135
  C:3860H         LINE#         136
  C:3862H         LINE#         185
  C:3865H         LINE#         196
  -------         ENDMOD        ?C_STARTUP

  -------         MODULE        MAIN
  C:0000H         SYMBOL        _ICE_DUMMY_
  D:0090H         PUBLIC        P1
  D:00B0H         PUBLIC        P3
  C:3D5DH         PUBLIC        main
  X:00A8H         PUBLIC        ref
  C:3188H         PUBLIC        showimage
  C:3B39H         PUBLIC        jiance
  C:2815H         PUBLIC        xianshi
  B:00B0H.2       PUBLIC        key1
  B:00B0H.3       PUBLIC        key2
  -------         PROC          JIANCE
  C:3B39H         LINE#         20
  C:3B39H         LINE#         21
  C:3B39H         LINE#         22
  C:3B3FH         LINE#         23
  C:3B3FH         LINE#         24
  C:3B46H         LINE#         25
  C:3B4EH         LINE#         26
  C:3B57H         LINE#         27
  C:3B5AH         LINE#         28
  C:3B5DH         LINE#         29
  C:3B5DH         LINE#         30
  C:3B60H         LINE#         31
  C:3B60H         LINE#         32
  C:3B63H         LINE#         33
  C:3B66H         LINE#         34
  C:3B66H         LINE#         35
  C:3B6BH         LINE#         36
  C:3B6BH         LINE#         37
  C:3B70H         LINE#         38
  C:3B77H         LINE#         39
  C:3B7EH         LINE#         40
  C:3B85H         LINE#         41
  C:3B8CH         LINE#         42
  C:3B93H         LINE#         43
  C:3B96H         LINE#         44
  C:3B96H         LINE#         45
  C:3B96H         LINE#         46
  -------         ENDPROC       JIANCE
  -------         PROC          XIANSHI
  -------         DO            
  X:0006H         SYMBOL        lx
  X:0008H         SYMBOL        ly
  -------         ENDDO         
BL51 BANKED LINKER/LOCATER V6.22                                                      01/21/2022  11:45:08  PAGE 7


  C:2815H         LINE#         47
  C:2815H         LINE#         48
  C:2815H         LINE#         50
  C:281DH         LINE#         51
  C:2826H         LINE#         52
  C:282FH         LINE#         53
  C:283AH         LINE#         54
  C:284BH         LINE#         55
  C:2877H         LINE#         56
  C:28A3H         LINE#         57
  C:28B3H         LINE#         58
  C:28FBH         LINE#         59
  C:2909H         LINE#         60
  C:2955H         LINE#         61
  C:2965H         LINE#         62
  C:29ADH         LINE#         63
  C:29BBH         LINE#         64
  -------         ENDPROC       XIANSHI
  -------         PROC          SHOWIMAGE
  -------         DO            
  X:0000H         SYMBOL        i
  X:0002H         SYMBOL        j
  X:0004H         SYMBOL        k
  -------         ENDDO         
  C:3188H         LINE#         66
  C:3188H         LINE#         67
  C:3188H         LINE#         69
  C:318FH         LINE#         70
  C:3192H         LINE#         71
  C:319BH         LINE#         72
  C:319BH         LINE#         73
  C:31A2H         LINE#         74
  C:31A2H         LINE#         75
  C:31F6H         LINE#         76
  C:31FDH         LINE#         77
  C:31FDH         LINE#         78
  C:3203H         LINE#         79
  C:3203H         LINE#         80
  C:320AH         LINE#         82
  C:320AH         LINE#         83
  C:3234H         LINE#         84
  C:3253H         LINE#         85
  C:3275H         LINE#         86
  C:3297H         LINE#         87
  C:329CH         LINE#         88
  -------         ENDPROC       SHOWIMAGE
  -------         PROC          MAIN
  C:3D5DH         LINE#         89
  C:3D5DH         LINE#         90
  C:3D5DH         LINE#         91
  C:3D60H         LINE#         92
  C:3D63H         LINE#         93
  C:3D6AH         LINE#         94
  C:3D79H         LINE#         95
  C:3D7CH         LINE#         97
  C:3D7CH         LINE#         98
  C:3D7CH         LINE#         99
BL51 BANKED LINKER/LOCATER V6.22                                                      01/21/2022  11:45:08  PAGE 8


  C:3D82H         LINE#         100
  C:3D82H         LINE#         101
  C:3D85H         LINE#         102
  C:3D85H         LINE#         103
  C:3D8EH         LINE#         105
  -------         ENDPROC       MAIN
  -------         ENDMOD        MAIN

  -------         MODULE        LCD
  C:0000H         SYMBOL        _ICE_DUMMY_
  D:0080H         PUBLIC        P0
  D:0090H         PUBLIC        P1
  D:00A0H         PUBLIC        P2
  D:00B0H         PUBLIC        P3
  C:3488H         PUBLIC        _LCD_ShowNum
  C:2D90H         PUBLIC        Lcd_Init
  C:3E79H         PUBLIC        _LCD_WR_DATA8
  C:3E46H         PUBLIC        _LCD_WR_REG_DATA
  X:0082H         PUBLIC        HT
  C:3E5FH         PUBLIC        _LCD_WR_REG
  C:3B97H         PUBLIC        _LCD_Clear
  X:0084H         PUBLIC        VT
  C:396EH         PUBLIC        _LCD_Show2Num
  C:38E8H         PUBLIC        _LCD_Fill
  C:3CDAH         PUBLIC        _mypow
  C:261EH         PUBLIC        _Draw_Circle
  B:0090H.0       PUBLIC        LCD_CS
  B:00B0H.7       PUBLIC        LCD_RD
  C:2A07H         PUBLIC        _LCD_DrawLine
  C:3C1BH         PUBLIC        _LCD_DrawPoint
  C:37BBH         PUBLIC        _LCD_ShowString
  C:2BF8H         PUBLIC        _LCD_ShowChar
  C:3E3BH         PUBLIC        _LCD_WR_DATA
  B:00B0H.5       PUBLIC        LCD_RS
  X:0086H         PUBLIC        HDP
  B:00B0H.6       PUBLIC        LCD_WR
  C:3711H         PUBLIC        _LCD_DrawRectangle
  C:3642H         PUBLIC        _showhanzi
  C:3C45H         PUBLIC        _LCD_DrawPoint_big
  C:3E54H         PUBLIC        _LCD_Writ_Bus
  X:0088H         PUBLIC        FPS
  X:008AH         PUBLIC        VDP
  X:008CH         PUBLIC        HPS
  X:008EH         PUBLIC        POINT_COLOR
  X:0090H         PUBLIC        HPW
  X:0091H         PUBLIC        LPS
  X:0093H         PUBLIC        BACK_COLOR
  B:0090H.2       PUBLIC        LCD_REST
  C:3D23H         PUBLIC        _Address_set
  X:0095H         PUBLIC        VPS
  X:0097H         PUBLIC        VPW
  -------         PROC          _LCD_WRIT_BUS
  D:0007H         SYMBOL        VH
  D:0005H         SYMBOL        VL
  C:3E54H         LINE#         30
  C:3E54H         LINE#         31
  C:3E54H         LINE#         32
BL51 BANKED LINKER/LOCATER V6.22                                                      01/21/2022  11:45:08  PAGE 9


  C:3E56H         LINE#         33
  C:3E5AH         LINE#         34
  C:3E5CH         LINE#         35
  C:3E5EH         LINE#         36
  -------         ENDPROC       _LCD_WRIT_BUS
  -------         PROC          _LCD_WR_DATA8
  D:0007H         SYMBOL        VH
  D:0005H         SYMBOL        VL
  C:3E79H         LINE#         48
  C:3E79H         LINE#         49
  C:3E79H         LINE#         50
  C:3E7BH         LINE#         51
  -------         ENDPROC       _LCD_WR_DATA8
  C:3E32H         SYMBOL        L?0111
  C:3E33H         SYMBOL        L?0112
  -------         PROC          L?0110
  -------         ENDPROC       L?0110
  C:3E32H         SYMBOL        L?0111
  C:3E33H         SYMBOL        L?0112
  -------         PROC          _LCD_WR_DATA
  D:0004H         SYMBOL        da
  C:3E3BH         LINE#         53
  C:3E3FH         LINE#         54
  C:3E3FH         LINE#         55
  C:3E41H         LINE#         56
  -------         ENDPROC       _LCD_WR_DATA
  -------         PROC          _LCD_WR_REG
  D:0004H         SYMBOL        da
  C:3E5FH         LINE#         58
  C:3E63H         LINE#         59
  C:3E63H         LINE#         60
  C:3E65H         LINE#         61
  -------         ENDPROC       _LCD_WR_REG
  -------         PROC          _LCD_WR_REG_DATA
  D:0006H         SYMBOL        reg
  D:0002H         SYMBOL        da
  C:3E46H         LINE#         63
  C:3E4AH         LINE#         64
  C:3E4AH         LINE#         65
  C:3E4DH         LINE#         66
  -------         ENDPROC       _LCD_WR_REG_DATA
  -------         PROC          _ADDRESS_SET
  X:0063H         SYMBOL        x1
  X:0065H         SYMBOL        y1
  D:0002H         SYMBOL        x2
  X:0069H         SYMBOL        y2
  C:3D23H         LINE#         68
  C:3D31H         LINE#         69
  C:3D31H         LINE#         70
  C:3D38H         LINE#         71
  C:3D3BH         LINE#         72
  C:3D3EH         LINE#         73
  C:3D43H         LINE#         74
  C:3D4AH         LINE#         75
  C:3D4FH         LINE#         76
  C:3D4FH         LINE#         77
  C:3D52H         LINE#         78
BL51 BANKED LINKER/LOCATER V6.22                                                      01/21/2022  11:45:08  PAGE 10


  C:3D55H         LINE#         79
  C:3D58H         LINE#         80
  -------         ENDPROC       _ADDRESS_SET
  -------         PROC          LCD_INIT
  C:2D90H         LINE#         82
  C:2D90H         LINE#         83
  C:2D90H         LINE#         86
  C:2D92H         LINE#         87
  C:2D95H         LINE#         88
  C:2D95H         LINE#         89
  C:2D9DH         LINE#         90
  C:2DABH         LINE#         91
  C:2DC1H         LINE#         92
  C:2DCFH         LINE#         93
  C:2DD7H         LINE#         94
  C:2DE7H         LINE#         95
  C:2DF0H         LINE#         96
  C:2DF0H         LINE#         97
  C:2DF2H         LINE#         98
  C:2DF4H         LINE#         99
  C:2DF6H         LINE#         100
  C:2DFDH         LINE#         101
  C:2DFFH         LINE#         102
  C:2E06H         LINE#         103
  C:2E08H         LINE#         105
  C:2E0FH         LINE#         106
  C:2E14H         LINE#         107
  C:2E19H         LINE#         108
  C:2E1EH         LINE#         109
  C:2E23H         LINE#         110
  C:2E28H         LINE#         111
  C:2E2DH         LINE#         112
  C:2E34H         LINE#         113
  C:2E39H         LINE#         114
  C:2E3EH         LINE#         115
  C:2E45H         LINE#         116
  C:2E4AH         LINE#         117
  C:2E51H         LINE#         118
  C:2E56H         LINE#         119
  C:2E5BH         LINE#         120
  C:2E60H         LINE#         122
  C:2E65H         LINE#         123
  C:2E6AH         LINE#         124
  C:2E6FH         LINE#         125
  C:2E72H         LINE#         126
  C:2E75H         LINE#         127
  C:2E78H         LINE#         128
  C:2E7BH         LINE#         129
  C:2E80H         LINE#         131
  C:2E85H         LINE#         132
  C:2E88H         LINE#         133
  C:2E8BH         LINE#         134
  C:2E8EH         LINE#         135
  C:2E91H         LINE#         136
  C:2E99H         LINE#         137
  C:2E99H         LINE#         138
  C:2E9CH         LINE#         139
BL51 BANKED LINKER/LOCATER V6.22                                                      01/21/2022  11:45:08  PAGE 11


  C:2EA1H         LINE#         141
  C:2EA6H         LINE#         142
  C:2EA9H         LINE#         143
  C:2EACH         LINE#         144
  C:2EB4H         LINE#         145
  C:2EB4H         LINE#         146
  C:2EB7H         LINE#         147
  C:2EBAH         LINE#         148
  C:2EBDH         LINE#         150
  C:2EC2H         LINE#         151
  C:2EC7H         LINE#         153
  C:2ECCH         LINE#         154
  C:2ED1H         LINE#         155
  C:2ED6H         LINE#         157
  C:2EDBH         LINE#         158
  C:2EE0H         LINE#         160
  C:2EE5H         LINE#         161
  C:2EEAH         LINE#         164
  C:2EEFH         LINE#         166
  C:2EF6H         LINE#         170
  C:2EFBH         LINE#         171
  -------         ENDPROC       LCD_INIT
  -------         PROC          _LCD_CLEAR
  D:0004H         SYMBOL        Color
  -------         DO            
  X:004AH         SYMBOL        VH
  D:0001H         SYMBOL        VL
  X:004BH         SYMBOL        i
  D:0002H         SYMBOL        j
  -------         ENDDO         
  C:3B97H         LINE#         177
  C:3B99H         LINE#         178
  C:3B99H         LINE#         181
  C:3B9EH         LINE#         182
  C:3BA0H         LINE#         183
  C:3BB6H         LINE#         184
  C:3BBDH         LINE#         185
  C:3BBDH         LINE#         186
  C:3BC0H         LINE#         187
  C:3BC0H         LINE#         188
  C:3BCAH         LINE#         189
  C:3BD5H         LINE#         191
  C:3BF2H         LINE#         192
  -------         ENDPROC       _LCD_CLEAR
  -------         PROC          _SHOWHANZI
  X:000AH         SYMBOL        x
  X:000CH         SYMBOL        y
  X:000EH         SYMBOL        index
  -------         DO            
  X:000FH         SYMBOL        i
  X:0010H         SYMBOL        j
  X:0011H         SYMBOL        temp
  -------         ENDDO         
  C:3642H         LINE#         195
  C:3657H         LINE#         196
  C:3657H         LINE#         198
  C:3665H         LINE#         199
BL51 BANKED LINKER/LOCATER V6.22                                                      01/21/2022  11:45:08  PAGE 12


  C:3691H         LINE#         200
  C:36A4H         LINE#         201
  C:36A9H         LINE#         202
  C:36A9H         LINE#         203
  C:36B8H         LINE#         204
  C:36B8H         LINE#         205
  C:36E2H         LINE#         206
  C:36E2H         LINE#         207
  C:36E5H         LINE#         208
  C:36E7H         LINE#         210
  C:36E7H         LINE#         211
  C:36F2H         LINE#         212
  C:36F2H         LINE#         213
  C:36FAH         LINE#         214
  C:3704H         LINE#         215
  C:3710H         LINE#         216
  -------         ENDPROC       _SHOWHANZI
  C:3C06H         SYMBOL        L?0114
  C:3C09H         SYMBOL        L?0115
  C:3C0AH         SYMBOL        L?0116
  -------         PROC          L?0113
  -------         ENDPROC       L?0113
  C:3C06H         SYMBOL        L?0114
  C:3C09H         SYMBOL        L?0115
  C:3C0AH         SYMBOL        L?0116
  -------         PROC          _LCD_DRAWPOINT
  D:0002H         SYMBOL        x
  D:0082H         SYMBOL        y
  C:3C1BH         LINE#         219
  C:3C23H         LINE#         220
  C:3C23H         LINE#         221
  C:3C3AH         LINE#         222
  -------         ENDPROC       _LCD_DRAWPOINT
  -------         PROC          _LCD_DRAWPOINT_BIG
  D:0002H         SYMBOL        x
  D:0082H         SYMBOL        y
  C:3C45H         LINE#         226
  C:3C4DH         LINE#         227
  C:3C4DH         LINE#         228
  -------         ENDPROC       _LCD_DRAWPOINT_BIG
  -------         PROC          _LCD_FILL
  X:000AH         SYMBOL        xsta
  X:000CH         SYMBOL        ysta
  X:000EH         SYMBOL        xend
  X:0010H         SYMBOL        yend
  X:0012H         SYMBOL        color
  -------         DO            
  X:0014H         SYMBOL        i
  D:0002H         SYMBOL        j
  -------         ENDDO         
  C:38E8H         LINE#         233
  C:38FCH         LINE#         234
  C:38FCH         LINE#         236
  C:3910H         LINE#         237
  C:3934H         LINE#         238
  C:3934H         LINE#         239
  C:395DH         LINE#         240
BL51 BANKED LINKER/LOCATER V6.22                                                      01/21/2022  11:45:08  PAGE 13


  C:396DH         LINE#         241
  -------         ENDPROC       _LCD_FILL
  -------         PROC          _LCD_DRAWLINE
  X:0047H         SYMBOL        x1
  X:0049H         SYMBOL        y1
  D:0002H         SYMBOL        x2
  X:004DH         SYMBOL        y2
  -------         DO            
  X:004FH         SYMBOL        t
  X:0051H         SYMBOL        xerr
  X:0053H         SYMBOL        yerr
  X:0055H         SYMBOL        delta_x
  X:0057H         SYMBOL        delta_y
  X:0059H         SYMBOL        distance
  X:005BH         SYMBOL        incx
  X:005DH         SYMBOL        incy
  X:005FH         SYMBOL        uRow
  X:0061H         SYMBOL        uCol
  -------         ENDDO         
  C:2A07H         LINE#         245
  C:2A15H         LINE#         246
  C:2A15H         LINE#         248
  C:2A20H         LINE#         251
  C:2A35H         LINE#         252
  C:2A50H         LINE#         253
  C:2A5FH         LINE#         254
  C:2A65H         LINE#         255
  C:2A81H         LINE#         256
  C:2A8DH         LINE#         257
  C:2AA2H         LINE#         258
  C:2ABEH         LINE#         259
  C:2ACAH         LINE#         260
  C:2ADFH         LINE#         261
  C:2B05H         LINE#         262
  C:2B0AH         LINE#         263
  C:2B2FH         LINE#         264
  C:2B2FH         LINE#         265
  C:2B40H         LINE#         266
  C:2B54H         LINE#         267
  C:2B68H         LINE#         268
  C:2B84H         LINE#         269
  C:2B84H         LINE#         270
  C:2B90H         LINE#         271
  C:2BA4H         LINE#         272
  C:2BA4H         LINE#         273
  C:2BC0H         LINE#         274
  C:2BC0H         LINE#         275
  C:2BCCH         LINE#         276
  C:2BE0H         LINE#         277
  C:2BE0H         LINE#         278
  C:2BF1H         LINE#         279
  -------         ENDPROC       _LCD_DRAWLINE
  -------         PROC          _LCD_DRAWRECTANGLE
  X:0000H         SYMBOL        x1
  X:0002H         SYMBOL        y1
  X:0004H         SYMBOL        x2
  X:0006H         SYMBOL        y2
BL51 BANKED LINKER/LOCATER V6.22                                                      01/21/2022  11:45:08  PAGE 14


  C:3711H         LINE#         281
  C:3727H         LINE#         282
  C:3727H         LINE#         283
  C:3743H         LINE#         284
  C:376AH         LINE#         285
  C:3792H         LINE#         286
  -------         ENDPROC       _LCD_DRAWRECTANGLE
  -------         PROC          _DRAW_CIRCLE
  X:0000H         SYMBOL        x0
  X:0002H         SYMBOL        y0
  D:0003H         SYMBOL        r
  -------         DO            
  X:0004H         SYMBOL        a
  X:0006H         SYMBOL        b
  X:0008H         SYMBOL        di
  -------         ENDDO         
  C:261EH         LINE#         291
  C:262CH         LINE#         292
  C:262CH         LINE#         295
  C:263BH         LINE#         296
  C:264FH         LINE#         297
  C:266DH         LINE#         298
  C:266DH         LINE#         299
  C:2692H         LINE#         300
  C:26BEH         LINE#         301
  C:26D5H         LINE#         302
  C:2702H         LINE#         303
  C:272FH         LINE#         304
  C:2748H         LINE#         305
  C:2774H         LINE#         306
  C:2777H         LINE#         307
  C:2792H         LINE#         308
  C:27A0H         LINE#         310
  C:27CFH         LINE#         312
  C:27CFH         LINE#         313
  C:2800H         LINE#         314
  C:280EH         LINE#         315
  C:280EH         LINE#         316
  C:2811H         LINE#         317
  C:2814H         LINE#         318
  -------         ENDPROC       _DRAW_CIRCLE
  -------         PROC          L?0117
  -------         ENDPROC       L?0117
  -------         PROC          _LCD_SHOWCHAR
  X:004FH         SYMBOL        x
  X:0051H         SYMBOL        y
  X:0053H         SYMBOL        num
  X:0054H         SYMBOL        mode
  -------         DO            
  X:0055H         SYMBOL        temp
  D:0001H         SYMBOL        pos
  X:0056H         SYMBOL        t
  X:0057H         SYMBOL        x0
  X:0059H         SYMBOL        colortemp
  -------         ENDDO         
  C:2BF8H         LINE#         328
  C:2C09H         LINE#         329
BL51 BANKED LINKER/LOCATER V6.22                                                      01/21/2022  11:45:08  PAGE 15


  C:2C09H         LINE#         332
  C:2C19H         LINE#         333
  C:2C28H         LINE#         334
  C:2C46H         LINE#         336
  C:2C4DH         LINE#         337
  C:2C79H         LINE#         338
  C:2C82H         LINE#         339
  C:2C82H         LINE#         340
  C:2C83H         LINE#         341
  C:2C83H         LINE#         342
  C:2CA5H         LINE#         343
  C:2CA8H         LINE#         344
  C:2CA8H         LINE#         345
  C:2CB4H         LINE#         346
  C:2CC3H         LINE#         347
  C:2CCEH         LINE#         348
  C:2CD5H         LINE#         349
  C:2CE3H         LINE#         350
  C:2CEFH         LINE#         351
  C:2CFEH         LINE#         352
  C:2D0CH         LINE#         353
  C:2D17H         LINE#         354
  C:2D17H         LINE#         355
  C:2D17H         LINE#         356
  C:2D19H         LINE#         357
  C:2D19H         LINE#         358
  C:2D3BH         LINE#         359
  C:2D48H         LINE#         360
  C:2D48H         LINE#         361
  C:2D6EH         LINE#         362
  C:2D75H         LINE#         363
  C:2D7BH         LINE#         364
  C:2D80H         LINE#         365
  C:2D80H         LINE#         366
  C:2D8FH         LINE#         367
  -------         ENDPROC       _LCD_SHOWCHAR
  -------         PROC          _MYPOW
  X:004FH         SYMBOL        m
  X:0050H         SYMBOL        n
  -------         DO            
  X:0051H         SYMBOL        result
  -------         ENDDO         
  C:3CDAH         LINE#         369
  C:3CE2H         LINE#         370
  C:3CE2H         LINE#         371
  C:3CEAH         LINE#         372
  C:3D14H         LINE#         373
  C:3D22H         LINE#         374
  -------         ENDPROC       _MYPOW
  -------         PROC          _LCD_SHOWNUM
  X:0043H         SYMBOL        x
  X:0045H         SYMBOL        y
  X:0047H         SYMBOL        num
  X:004BH         SYMBOL        len
  -------         DO            
  X:004CH         SYMBOL        t
  X:004DH         SYMBOL        temp
BL51 BANKED LINKER/LOCATER V6.22                                                      01/21/2022  11:45:08  PAGE 16


  X:004EH         SYMBOL        enshow
  -------         ENDDO         
  C:3488H         LINE#         380
  C:3496H         LINE#         381
  C:3496H         LINE#         383
  C:349BH         LINE#         384
  C:34AEH         LINE#         385
  C:34C2H         LINE#         386
  C:34C2H         LINE#         387
  C:34F3H         LINE#         388
  C:3504H         LINE#         389
  C:3504H         LINE#         390
  C:3508H         LINE#         391
  C:3508H         LINE#         392
  C:352AH         LINE#         393
  C:352CH         LINE#         394
  C:3532H         LINE#         396
  C:3532H         LINE#         397
  C:355FH         LINE#         398
  C:3568H         LINE#         399
  -------         ENDPROC       _LCD_SHOWNUM
  -------         PROC          _LCD_SHOW2NUM
  X:0000H         SYMBOL        x
  X:0002H         SYMBOL        y
  X:0004H         SYMBOL        num
  X:0006H         SYMBOL        len
  -------         DO            
  X:0007H         SYMBOL        t
  X:0008H         SYMBOL        temp
  -------         ENDDO         
  C:396EH         LINE#         403
  C:3982H         LINE#         404
  C:3982H         LINE#         406
  C:3993H         LINE#         407
  C:3993H         LINE#         408
  C:39C3H         LINE#         409
  C:39E7H         LINE#         410
  C:39EFH         LINE#         411
  -------         ENDPROC       _LCD_SHOW2NUM
  -------         PROC          _LCD_SHOWSTRING
  X:0043H         SYMBOL        x
  X:0045H         SYMBOL        y
  X:0047H         SYMBOL        p
  C:37BBH         LINE#         416
  C:37D2H         LINE#         417
  C:37D2H         LINE#         418
  C:37E2H         LINE#         419
  C:37E2H         LINE#         420
  C:3803H         LINE#         421
  C:3823H         LINE#         422
  C:3840H         LINE#         423
  C:384EH         LINE#         424
  C:3858H         LINE#         425
  C:385BH         LINE#         426
  -------         ENDPROC       _LCD_SHOWSTRING
  -------         ENDMOD        LCD

BL51 BANKED LINKER/LOCATER V6.22                                                      01/21/2022  11:45:08  PAGE 17


  -------         MODULE        SYS
  C:0000H         SYMBOL        _ICE_DUMMY_
  C:3DB9H         PUBLIC        _delayms
  -------         PROC          _DELAYMS
  D:0006H         SYMBOL        count
  -------         DO            
  D:0004H         SYMBOL        i
  D:0002H         SYMBOL        j
  -------         ENDDO         
  C:3DB9H         LINE#         4
  C:3DB9H         LINE#         5
  C:3DB9H         LINE#         7
  C:3DC9H         LINE#         8
  C:3DDEH         LINE#         9
  -------         ENDPROC       _DELAYMS
  -------         ENDMOD        SYS

  -------         MODULE        FONT
  C:0000H         SYMBOL        _ICE_DUMMY_
  C:0003H         PUBLIC        image
  C:0D83H         PUBLIC        asc2_1608
  C:0C83H         PUBLIC        hanzi
  -------         ENDMOD        FONT

  -------         MODULE        TOUCH
  C:0000H         SYMBOL        _ICE_DUMMY_
  D:0090H         PUBLIC        P1
  D:00B0H         PUBLIC        P3
  C:3DDFH         PUBLIC        ReadFromCharFrom7843
  C:3E73H         PUBLIC        tpstate
  C:3E6AH         PUBLIC        spistar
  B:0090H.4       PUBLIC        CS
  B:00D0H.7       PUBLIC        CY
  C:3E1BH         PUBLIC        _ADS_Read_AD
  B:0090H.7       PUBLIC        DCLK
  C:3E01H         PUBLIC        _WriteCharTo7843
  C:3569H         PUBLIC        point
  C:3AD6H         PUBLIC        _Read_ADS
  B:00B0H.1       PUBLIC        DOUT
  X:0098H         PUBLIC        chx
  X:009AH         PUBLIC        chy
  C:2F00H         PUBLIC        _ADS_Read_XY
  X:009CH         PUBLIC        tp_pixlcd
  C:1373H         PUBLIC        Touch_Adjust
  B:00B0H.0       PUBLIC        DIN
  X:00A0H         PUBLIC        tp_pixad
  C:3057H         PUBLIC        _Read_ADS2
  C:39F0H         PUBLIC        Read_TP_Once
  X:00A4H         PUBLIC        vx
  X:00A6H         PUBLIC        vy
  C:33A0H         PUBLIC        _Drow_Touch_Point
  B:00B0H.4       PUBLIC        Penirq
  C:329DH         PUBLIC        Convert_Pos
  -------         PROC          TPSTATE
  C:3E73H         LINE#         15
  C:3E73H         LINE#         16
  C:3E73H         LINE#         17
BL51 BANKED LINKER/LOCATER V6.22                                                      01/21/2022  11:45:08  PAGE 18


  C:3E78H         LINE#         18
  -------         ENDPROC       TPSTATE
  -------         PROC          SPISTAR
  C:3E6AH         LINE#         20
  C:3E6AH         LINE#         21
  C:3E6AH         LINE#         22
  C:3E6CH         LINE#         23
  C:3E6EH         LINE#         24
  C:3E70H         LINE#         25
  C:3E72H         LINE#         26
  -------         ENDPROC       SPISTAR
  -------         PROC          _WRITECHARTO7843
  D:0007H         SYMBOL        num
  -------         DO            
  D:0006H         SYMBOL        count
  -------         ENDDO         
  C:3E01H         LINE#         28
  C:3E01H         LINE#         29
  C:3E01H         LINE#         30
  C:3E03H         LINE#         31
  C:3E05H         LINE#         32
  C:3E05H         LINE#         33
  C:3E05H         LINE#         34
  C:3E09H         LINE#         35
  C:3E0BH         LINE#         36
  C:3E10H         LINE#         37
  C:3E15H         LINE#         38
  C:3E1AH         LINE#         39
  -------         ENDPROC       _WRITECHARTO7843
  -------         PROC          READFROMCHARFROM7843
  -------         DO            
  D:0005H         SYMBOL        count
  D:0006H         SYMBOL        Num
  -------         ENDDO         
  C:3DDFH         LINE#         41
  C:3DDFH         LINE#         42
  C:3DDFH         LINE#         43
  C:3DE1H         LINE#         44
  C:3DE3H         LINE#         45
  C:3DE3H         LINE#         46
  C:3DE3H         LINE#         47
  C:3DEAH         LINE#         48
  C:3DEFH         LINE#         49
  C:3DF4H         LINE#         50
  C:3DF7H         LINE#         51
  C:3DF7H         LINE#         52
  C:3DFBH         LINE#         53
  C:3DFBH         LINE#         55
  C:3E00H         LINE#         57
  C:3E00H         LINE#         58
  -------         ENDPROC       READFROMCHARFROM7843
  -------         PROC          _ADS_READ_AD
  D:0007H         SYMBOL        CMD
  -------         DO            
  D:0006H         SYMBOL        l
  -------         ENDDO         
  C:3E1BH         LINE#         60
BL51 BANKED LINKER/LOCATER V6.22                                                      01/21/2022  11:45:08  PAGE 19


  C:3E1BH         LINE#         61
  C:3E1BH         LINE#         63
  C:3E1DH         LINE#         64
  C:3E20H         LINE#         65
  C:3E26H         LINE#         66
  C:3E2CH         LINE#         67
  C:3E2FH         LINE#         68
  C:3E31H         LINE#         69
  C:3E31H         LINE#         70
  -------         ENDPROC       _ADS_READ_AD
  -------         PROC          _ADS_READ_XY
  D:0001H         SYMBOL        xy
  -------         DO            
  D:0002H         SYMBOL        i
  X:005EH         SYMBOL        j
  X:0060H         SYMBOL        buf
  X:007EH         SYMBOL        sum
  X:0080H         SYMBOL        temp
  -------         ENDDO         
  C:2F00H         LINE#         76
  C:2F02H         LINE#         77
  C:2F02H         LINE#         80
  C:2F09H         LINE#         82
  C:2F0BH         LINE#         83
  C:2F0BH         LINE#         84
  C:2F2AH         LINE#         85
  C:2F35H         LINE#         86
  C:2F38H         LINE#         87
  C:2F38H         LINE#         88
  C:2F58H         LINE#         89
  C:2F58H         LINE#         90
  C:2F8AH         LINE#         91
  C:2F8AH         LINE#         92
  C:2F92H         LINE#         93
  C:2FC4H         LINE#         94
  C:2FE8H         LINE#         95
  C:2FE8H         LINE#         96
  C:2FFCH         LINE#         97
  C:300AH         LINE#         98
  C:3011H         LINE#         99
  C:3041H         LINE#         100
  C:3056H         LINE#         101
  C:3056H         LINE#         102
  -------         ENDPROC       _ADS_READ_XY
  -------         PROC          _READ_ADS
  X:0056H         SYMBOL        x
  X:0059H         SYMBOL        y
  -------         DO            
  X:005CH         SYMBOL        xtemp
  D:0006H         SYMBOL        ytemp
  -------         ENDDO         
  C:3AD6H         LINE#         105
  C:3AE1H         LINE#         106
  C:3AE1H         LINE#         108
  C:3AEEH         LINE#         109
  C:3AF3H         LINE#         110
  C:3B0DH         LINE#         111
BL51 BANKED LINKER/LOCATER V6.22                                                      01/21/2022  11:45:08  PAGE 20


  C:3B25H         LINE#         112
  C:3B36H         LINE#         113
  C:3B38H         LINE#         114
  -------         ENDPROC       _READ_ADS
  -------         PROC          _READ_ADS2
  X:0048H         SYMBOL        x
  X:004BH         SYMBOL        y
  -------         DO            
  X:004EH         SYMBOL        x1
  X:0050H         SYMBOL        y1
  X:0052H         SYMBOL        x2
  X:0054H         SYMBOL        y2
  D:0007H         SYMBOL        flag
  -------         ENDDO         
  C:3057H         LINE#         119
  C:3062H         LINE#         120
  C:3062H         LINE#         124
  C:3079H         LINE#         125
  C:307EH         LINE#         126
  C:3095H         LINE#         127
  C:309AH         LINE#         128
  C:3130H         LINE#         130
  C:3130H         LINE#         131
  C:3159H         LINE#         132
  C:3182H         LINE#         133
  C:3185H         LINE#         134
  C:3187H         LINE#         135
  -------         ENDPROC       _READ_ADS2
  -------         PROC          READ_TP_ONCE
  -------         DO            
  X:0043H         SYMBOL        re
  X:0044H         SYMBOL        x1
  X:0046H         SYMBOL        y1
  -------         ENDDO         
  C:39F0H         LINE#         137
  C:39F0H         LINE#         138
  C:39F0H         LINE#         139
  C:39F5H         LINE#         141
  C:39FBH         LINE#         142
  C:39FBH         LINE#         143
  C:3A15H         LINE#         144
  C:3A1CH         LINE#         145
  C:3A36H         LINE#         146
  C:3A5EH         LINE#         147
  C:3A5EH         LINE#         148
  C:3A63H         LINE#         149
  C:3A63H         LINE#         150
  C:3A65H         LINE#         151
  C:3A6AH         LINE#         152
  -------         ENDPROC       READ_TP_ONCE
  -------         PROC          _DROW_TOUCH_POINT
  X:0043H         SYMBOL        x
  X:0045H         SYMBOL        y
  C:33A0H         LINE#         157
  C:33AEH         LINE#         158
  C:33AEH         LINE#         159
  C:33D8H         LINE#         160
BL51 BANKED LINKER/LOCATER V6.22                                                      01/21/2022  11:45:08  PAGE 21


  C:340CH         LINE#         161
  C:342BH         LINE#         162
  C:344AH         LINE#         163
  C:3469H         LINE#         164
  -------         ENDPROC       _DROW_TOUCH_POINT
  -------         PROC          CONVERT_POS
  -------         DO            
  X:000AH         SYMBOL        l
  -------         ENDDO         
  C:329DH         LINE#         169
  C:329DH         LINE#         170
  C:329DH         LINE#         171
  C:32A2H         LINE#         172
  C:32BEH         LINE#         173
  C:32BEH         LINE#         174
  C:32C4H         LINE#         175
  C:332FH         LINE#         176
  C:339AH         LINE#         177
  C:339AH         LINE#         178
  C:339FH         LINE#         179
  -------         ENDPROC       CONVERT_POS
  -------         PROC          TOUCH_ADJUST
  -------         DO            
  X:0006H         SYMBOL        vx1
  X:000AH         SYMBOL        vx2
  X:000EH         SYMBOL        vy1
  X:0012H         SYMBOL        vy2
  X:0016H         SYMBOL        chx1
  X:0018H         SYMBOL        chx2
  X:001AH         SYMBOL        chy1
  X:001CH         SYMBOL        chy2
  X:001EH         SYMBOL        lx
  X:0020H         SYMBOL        ly
  X:0022H         SYMBOL        p
  X:0042H         SYMBOL        cnt
  -------         ENDDO         
  C:1373H         LINE#         184
  C:1373H         LINE#         185
  C:1373H         LINE#         190
  C:1378H         LINE#         191
  C:1379H         LINE#         192
  C:1381H         LINE#         193
  C:1389H         LINE#         194
  C:138EH         LINE#         195
  C:1396H         LINE#         196
  C:1396H         LINE#         197
  C:1399H         LINE#         198
  C:1399H         LINE#         199
  C:1399H         LINE#         200
  C:139CH         LINE#         201
  C:139CH         LINE#         202
  C:13A2H         LINE#         203
  C:13A2H         LINE#         204
  C:13C2H         LINE#         205
  C:13DEH         LINE#         206
  C:13E4H         LINE#         207
  C:13E4H         LINE#         208
BL51 BANKED LINKER/LOCATER V6.22                                                      01/21/2022  11:45:08  PAGE 22


  C:13F6H         LINE#         209
  C:13F6H         LINE#         210
  C:13F6H         LINE#         211
  C:13FDH         LINE#         212
  C:1400H         LINE#         213
  C:1400H         LINE#         214
  C:1400H         LINE#         215
  C:1404H         LINE#         216
  C:1406H         LINE#         217
  C:1406H         LINE#         218
  C:140DH         LINE#         219
  C:1410H         LINE#         220
  C:1410H         LINE#         221
  C:1410H         LINE#         222
  C:1414H         LINE#         223
  C:1417H         LINE#         224
  C:1417H         LINE#         225
  C:141EH         LINE#         226
  C:1421H         LINE#         227
  C:1421H         LINE#         228
  C:1421H         LINE#         229
  C:1429H         LINE#         230
  C:142CH         LINE#         231
  C:142CH         LINE#         232
  C:1433H         LINE#         233
  C:1436H         LINE#         234
  C:1436H         LINE#         235
  C:1436H         LINE#         236
  C:14E1H         LINE#         237
  C:1589H         LINE#         238
  C:161DH         LINE#         239
  C:16C5H         LINE#         241
  C:1770H         LINE#         242
  C:1818H         LINE#         243
  C:18ACH         LINE#         244
  C:1954H         LINE#         247
  C:1A92H         LINE#         248
  C:1A92H         LINE#         249
  C:1A97H         LINE#         250
  C:1A9EH         LINE#         251
  C:1AA9H         LINE#         252
  C:1AACH         LINE#         253
  C:1AACH         LINE#         254
  C:1B12H         LINE#         255
  C:1B54H         LINE#         258
  C:1B5BH         LINE#         259
  C:1B62H         LINE#         260
  C:1B6AH         LINE#         262
  C:1B77H         LINE#         263
  C:1BC4H         LINE#         264
  C:1BD9H         LINE#         265
  C:1C28H         LINE#         266
  C:1C3DH         LINE#         267
  C:1C86H         LINE#         268
  C:1C9BH         LINE#         269
  C:1CE4H         LINE#         271
  C:1CF4H         LINE#         272
BL51 BANKED LINKER/LOCATER V6.22                                                      01/21/2022  11:45:08  PAGE 23


  C:1D42H         LINE#         273
  C:1D59H         LINE#         274
  C:1DA9H         LINE#         275
  C:1DC0H         LINE#         276
  C:1E0AH         LINE#         277
  C:1E21H         LINE#         278
  C:1E6BH         LINE#         280
  C:1E7BH         LINE#         281
  C:1EC3H         LINE#         282
  C:1EDAH         LINE#         283
  C:1F24H         LINE#         284
  C:1F3BH         LINE#         285
  C:1F85H         LINE#         286
  C:1F9CH         LINE#         287
  C:1FE6H         LINE#         289
  C:1FFDH         LINE#         290
  C:200FH         LINE#         291
  C:2012H         LINE#         293
  C:2019H         LINE#         295
  C:2019H         LINE#         296
  C:2019H         LINE#         297
  C:2019H         LINE#         298
  -------         ENDPROC       TOUCH_ADJUST
  -------         PROC          POINT
  -------         DO            
  X:0006H         SYMBOL        t
  -------         ENDDO         
  C:3569H         LINE#         299
  C:3569H         LINE#         300
  C:3569H         LINE#         301
  C:3573H         LINE#         303
  C:3573H         LINE#         304
  C:3573H         LINE#         305
  C:3579H         LINE#         306
  C:3579H         LINE#         307
  C:3583H         LINE#         308
  C:3589H         LINE#         309
  C:3589H         LINE#         312
  C:35BCH         LINE#         313
  C:35EFH         LINE#         314
  C:3600H         LINE#         315
  C:3600H         LINE#         317
  C:3603H         LINE#         319
  C:3603H         LINE#         320
  C:3621H         LINE#         321
  C:3641H         LINE#         322
  -------         ENDPROC       POINT
  -------         ENDMOD        TOUCH

  -------         MODULE        ?C?FPADD
  C:2021H         PUBLIC        ?C?FPADD
  C:201DH         PUBLIC        ?C?FPSUB
  -------         ENDMOD        ?C?FPADD

  -------         MODULE        ?C?FPMUL
  C:2112H         PUBLIC        ?C?FPMUL
  -------         ENDMOD        ?C?FPMUL
BL51 BANKED LINKER/LOCATER V6.22                                                      01/21/2022  11:45:08  PAGE 24



  -------         MODULE        ?C?FPDIV
  C:221BH         PUBLIC        ?C?FPDIV
  -------         ENDMOD        ?C?FPDIV

  -------         MODULE        ?C?FPCMP
  C:22BAH         PUBLIC        ?C?FPCMP
  C:22B8H         PUBLIC        ?C?FPCMP3
  -------         ENDMOD        ?C?FPCMP

  -------         MODULE        ?C?FCAST
  C:233BH         PUBLIC        ?C?FCASTC
  C:2336H         PUBLIC        ?C?FCASTI
  C:2331H         PUBLIC        ?C?FCASTL
  -------         ENDMOD        ?C?FCAST

  -------         MODULE        ?C?CASTF
  C:236FH         PUBLIC        ?C?CASTF
  -------         ENDMOD        ?C?CASTF

  -------         MODULE        ?C?CLDPTR
  C:23F0H         PUBLIC        ?C?CLDPTR
  -------         ENDMOD        ?C?CLDPTR

  -------         MODULE        ?C?IMUL
  C:2409H         PUBLIC        ?C?IMUL
  -------         ENDMOD        ?C?IMUL

  -------         MODULE        ?C?UIDIV
  C:241BH         PUBLIC        ?C?UIDIV
  -------         ENDMOD        ?C?UIDIV

  -------         MODULE        ?C?IILDX
  C:2470H         PUBLIC        ?C?IILDX
  -------         ENDMOD        ?C?IILDX

  -------         MODULE        ?C?ISTPTR
  C:2486H         PUBLIC        ?C?ISTPTR
  -------         ENDMOD        ?C?ISTPTR

  -------         MODULE        ?C?LMUL
  C:24A5H         PUBLIC        ?C?LMUL
  -------         ENDMOD        ?C?LMUL

  -------         MODULE        ?C?ULDIV
  C:2530H         PUBLIC        ?C?ULDIV
  -------         ENDMOD        ?C?ULDIV

  -------         MODULE        ?C?LNEG
  C:25C2H         PUBLIC        ?C?LNEG
  -------         ENDMOD        ?C?LNEG

  -------         MODULE        ?C?ULCMP
  C:25D0H         PUBLIC        ?C?ULCMP
  -------         ENDMOD        ?C?ULCMP

  -------         MODULE        ?C?LSTXDATA
BL51 BANKED LINKER/LOCATER V6.22                                                      01/21/2022  11:45:08  PAGE 25


  C:25E1H         PUBLIC        ?C?LSTXDATA
  -------         ENDMOD        ?C?LSTXDATA

  -------         MODULE        ?C?LSTKXDATA
  C:25EDH         PUBLIC        ?C?LSTKXDATA
  -------         ENDMOD        ?C?LSTKXDATA

Program Size: data=9.0 xdata=169 code=16000
LINK/LOCATE RUN COMPLETE.  0 WARNING(S),  0 ERROR(S)
